:100000000C9462000C948A000C948A000C948A0070
:100010000C948A000C948A000C948A000C948A0038
:100020000C948A000C948A000C948A000C948A0028
:100030000C948A000C948A000C948A000C948A0018
:100040000C9403030C948A000C942A040C948A00E8
:100050000C948A000C948A000C948A000C948A00F8
:100060000C948A000C948A000000000024002700F1
:100070002A0000000000250028002B0000000000DE
:1000800023002600290004040404040404040202DA
:100090000202020203030303030301020408102007
:1000A0004080010204081020010204081020000012
:1000B0000007000201000003040600000000000029
:1000C0000000730511241FBECFEFD8E0DEBFCDBF07
:1000D00011E0A0E0B1E0EEEDFCE002C005900D9271
:1000E000A231B107D9F711E0A2E1B1E001C01D9240
:1000F000AE3EB107E1F710E0C4ECD0E004C02297B7
:10010000FE010E946906C23CD107C9F70E94FC02A9
:100110000C946D060C940000CF92DF92FF920F9327
:100120001F93CF93DF93F82E062F142F862F61E0B5
:100130000E94BD038F2D61E00E94BD038F2D60E002
:100140000E94DD03802F60E00E94DD03C7E0D0E065
:10015000C12EDD24802F60E00E94DD03B6010C2E4D
:1001600002C0759567950A94E2F761708F2D0E9421
:10017000DD03802F61E00E94DD038F2D60E00E948F
:10018000DD0321978FEFCF3FD80721F7802F60E065
:100190000E94DD03DF91CF911F910F91FF90DF90BF
:1001A000CF900895AF92BF92CF92DF92EF92FF92DD
:1001B0000F931F93CF93DF935C018B01809100011C
:1001C00060E00E94DD036091020170910301809163
:1001D00004019091050140E00E948C0060910201B1
:1001E00070910301809104019091050140E00E940B
:1001F0008C008091000161E00E94DD0368EC70E0FA
:1002000080E090E00E945903C0E0D0E06801EE2455
:10021000D7FCE094FE2C75C08091000160E00E9444
:10022000DD036091020170910301809104019091BE
:1002300005014FEF0E948C00609102017091030153
:1002400080910401909105014FEF0E948C00609114
:1002500002017091030180910401909105014FEF1B
:100260000E948C0060910201709103018091040151
:10027000909105014FEF0E948C008091000161E098
:100280000E94DD03C701B6010E945903809100015D
:1002900060E00E94DD036091020170910301809192
:1002A00004019091050140E00E948C0060910201E0
:1002B00070910301809104019091050140E00E943A
:1002C0008C00609102017091030180910401909172
:1002D000050140E00E948C006091020170910301D1
:1002E000809104019091050140E00E948C00809172
:1002F000000161E00E94DD03C701B6010E945903BD
:100300002196CA15DB050CF487CFDF91CF911F91A1
:100310000F91FF90EF90DF90CF90BF90AF90089536
:10032000EF92FF920F931F93E0901201F090130150
:1003300000911401109115018091000160E00E946C
:10034000DD032091020130910301C8016AE070E0F1
:100350000E940306FB01E85EFE4F8091040190912C
:100360000501B90140810E948C0020910201309169
:100370000301C8016AE070E00E940306FC01EE5D23
:10038000FE4F8091040190910501B90140810E94C6
:100390008C002091020130910301C7016AE070E0F6
:1003A0000E940306FB01E45DFE4F809104019091E1
:1003B0000501B90140810E948C0020910201309119
:1003C0000301C7016AE070E00E940306FC01EA5CD9
:1003D000FE4F8091040190910501B90140810E9476
:1003E0008C008091000161E00E94DD031F910F915C
:1003F000FF90EF9008950E944B0320914A013091A5
:100400004B0140914C0150914D01621B730B840BC9
:10041000950B685E734080409040A8F00E944B03AB
:1004200060934A0170934B0180934C0190934D016E
:100430000E94900180911201909113010196909376
:100440001301809312018091120190911301CC97B6
:100450006CF0809114019091150101969093150113
:1004600080931401109213011092120180911401D3
:1004700090911501CC976CF0809116019091170125
:100480000196909317018093160110921501109216
:100490001401809116019091170148976CF080919A
:1004A0000601909107010196909307018093060140
:1004B0001092170110921601809106019091070188
:1004C000089734F081E090E0909307018093060153
:1004D00008958091000161E00E94BD038BED91E0E1
:1004E00040E855E260E070E00E9467048FE6809388
:1004F000180183E080931901FDE5F0931A0187E567
:1005000080931B0183E380931C0186E780931D0188
:100510008EE780931E0183E480931F01EFE7E09351
:10052000200177E7709321011092400181E08093D0
:100530004101109242018093430110924401809343
:100540004501109246018093470110924801809323
:1005500049018EED8093220186E0809323018AEB8E
:10056000809324018EEA8093250196E690932601DC
:100570008CEE809327018CEF8093280186E880938E
:1005800029018EEF80932A018EEE80932B016BE779
:1005900060932C0150E650932D01F0932E0145E716
:1005A00040932F019093300137E3309331012FE3D3
:1005B0002093320181E680933301E09334017093FC
:1005C00035016093360150933701F0933801409321
:1005D000390190933A0130933B0120933C01809381
:1005E0003D01E0933E0170933F0182E090E064EFB3
:1005F00071E00E94D20008950E9483030E94690264
:100600000E94FB01FDCF1F920F920FB60F92112493
:100610002F933F938F939F93AF93BF9380915201FA
:1006200090915301A0915401B09155013091560120
:100630000196A11DB11D232F2D5F2D3720F02D57C1
:100640000196A11DB11D20935601809352019093F4
:100650005301A0935401B093550180914E019091A4
:100660004F01A0915001B09151010196A11DB11D02
:1006700080934E0190934F01A0935001B09351018C
:10068000BF91AF919F918F913F912F910F900FBE8E
:100690000F901F9018958FB7F894209152013091C8
:1006A000530140915401509155018FBFB901CA01C6
:1006B0000895EF92FF920F931F937B018C018FB7E8
:1006C000F8944091520150915301609154017091FE
:1006D00055018FBF2FB7F89480915201909153012B
:1006E000A0915401B09155012FBF841B950BA60B0F
:1006F000B70BE816F9060A071B0760F71F910F9161
:10070000FF90EF900895789484B5826084BD84B59D
:10071000816084BD85B5826085BD85B5816085BDFC
:10072000EEE6F0E0808181608083E1E8F0E08081A6
:1007300082608083808181608083E0E8F0E0808156
:1007400081608083E1EBF0E0808184608083E0EB76
:10075000F0E0808181608083EAE7F0E0808184605E
:1007600080838081826080838081816080838081BA
:10077000806880831092C1000895282F30E0C9015D
:1007800086569F4FFC0194912A573F4FF90184915F
:10079000882391F0E82FF0E0EE0FFF1FE859FF4F9C
:1007A000A591B491662329F48C91909589238C931B
:1007B00008958C91892B8C930895482F50E0CA019D
:1007C00082559F4FFC012491CA0186569F4FFC0120
:1007D00094914A575F4FFA0134913323D1F1222388
:1007E00031F1233021F4809180008F7705C02430CF
:1007F00031F4809180008F7D8093800018C021307B
:1008000019F484B58F7704C0223021F484B58F7D2C
:1008100084BD0DC0263021F48091B0008F7705C0D3
:10082000273029F48091B0008F7D8093B000E32FB2
:10083000F0E0EE0FFF1FEE58FF4FA591B491662335
:1008400029F48C91909589238C9308958C91892B10
:100850008C9308951F920F920FB60F9211242F932D
:100860003F934F935F936F937F938F939F93AF9338
:10087000BF93EF93FF934091C600E091D701F091B1
:10088000D801CF01019660E870E00E9403069C0148
:100890008091D9019091DA012817390739F0E95A86
:1008A000FE4F40833093D8012093D701FF91EF9101
:1008B000BF91AF919F918F917F916F915F914F9178
:1008C0003F912F910F900FBE0F901F9018955F9240
:1008D0006F927F928F929F92AF92BF92CF92DF9250
:1008E000EF92FF920F931F93CF93DF93EC013A01A6
:1008F0004B01413482E458078FE0680780E07807B5
:100900000CF07FC060E874E88EE190E0A4019301F0
:100910000E9438062150304040405040CA01B90181
:1009200022E030E040E050E00E94380659016A01C0
:10093000A6019501209530954095509594E0220FA1
:10094000331F441F551F9A95D1F760E074E284EF7E
:1009500090E00E943806CA01B9012FEF30E040E074
:1009600050E00E94E405A40193010E943806C901E9
:1009700081509F4F181619061CF4522E5A9403C02A
:1009800055245394521A60E079E08DE390E0A4017D
:1009900093010E9438062150304040405040CA0127
:1009A000B90122E030E040E050E00E943806209596
:1009B00030954095509583E0220F331F441F551FFB
:1009C0008A95D1F760E074E284EF90E00E943806E7
:1009D000CA01B9012FEF30E040E050E00E94E40589
:1009E000A40193010E943806C90181509F4F181637
:1009F00019061CF4822F815002C081E0821B8515EC
:100A000000F5E885F98581E090E00A8802C0880F4A
:100A1000991F0A94E2F7808360E079E08DE390E02B
:100A2000A40193010E9438062150304040405040BC
:100A3000CA01B90122E030E040E050E00E943806EF
:100A400004C0E885F98510829501EC81FD81308331
:100A5000EE81FF812083EA85FB85208141E050E023
:100A6000CA010E8402C0880F991F0A94E2F7282B4E
:100A70002083EA85FB852081CA010F8402C0880F8C
:100A8000991F0A94E2F7282B2083EA85FB85808151
:100A9000088802C0440F551F0A94E2F7842B808314
:100AA000DF91CF911F910F91FF90EF90DF90CF904A
:100AB000BF90AF909F908F907F906F905F900895C0
:100AC000FC01A085B18521898C9190E0022E02C0A5
:100AD000959587950A94E2F780FFF6CF0484F58513
:100AE000E02D608308958CE091E09093DC01809389
:100AF000DB0187E591E09093DE018093DD0185ECD9
:100B000090E09093E0018093DF0184EC90E090937B
:100B1000E2018093E10180EC90E09093E401809306
:100B2000E30181EC90E09093E6018093E50186EC8F
:100B300090E09093E8018093E70184E08093E901DD
:100B400083E08093EA0187E08093EB0185E0809366
:100B5000EC0181E08093ED0108950F931F93CF93F3
:100B6000DF938C01EB0109C02196D801ED91FC9136
:100B70000190F081E02DC801099568816623A1F7F5
:100B8000DF91CF911F910F910895EF92FF920F93F4
:100B90001F93CF93DF938C017B01EA010CC0D70137
:100BA0006D917D01D801ED91FC910190F081E02DD6
:100BB000C80109952197209791F7DF91CF911F9157
:100BC0000F91FF90EF900895629FD001739FF00105
:100BD000829FE00DF11D649FE00DF11D929FF00DCD
:100BE000839FF00D749FF00D659FF00D9927729F04
:100BF000B00DE11DF91F639FB00DE11DF91FBD018F
:100C0000CF011124089597FB092E07260AD077FDFE
:100C100004D049D006D000201AF4709561957F4F1A
:100C20000895F6F7909581959F4F0895A1E21A2EA9
:100C3000AA1BBB1BFD010DC0AA1FBB1FEE1FFF1F80
:100C4000A217B307E407F50720F0A21BB30BE40BD0
:100C5000F50B661F771F881F991F1A9469F7609517
:100C60007095809590959B01AC01BD01CF010895D1
:100C700097FB092E05260ED057FD04D0D7DF0AD0EA
:100C8000001C38F450954095309521953F4F4F4FBB
:100C90005F4F0895F6F790958095709561957F4F19
:100CA0008F4F9F4F0895AA1BBB1B51E107C0AA1F7E
:100CB000BB1FA617B70710F0A61BB70B881F991FFD
:100CC0005A95A9F780959095BC01CD010895EE0F36
:0E0CD000FF1F0590F491E02D0994F894FFCFDA
:100CDE0008000C000B000100000000006005AD05CF
:020CEE00C5053A
:00000001FF
